:0200000480007A
:100000006F000005732F2034930F80006308FF03F7
:10001000930F90006304FF03930FB0006300FF038E
:10002000130F000063040F0067000F00732F2034CC
:1000300063540F006F00400093E19153171F0000BD
:1000400023223FFC171F000023200FFC6FF01FFF2F
:100050009300000013010000930100001302000050
:100060009302000013030000930300001304000038
:100070009304000013050000930500001306000020
:100080009306000013070000930700001308000008
:10009000930800001309000093090000130A0000F0
:1000A000930A0000130B0000930B0000130C0000D8
:1000B000930C0000130D0000930D0000130E0000C0
:1000C000930E0000130F0000930F0000732540F102
:1000D0006310050097020000938202017390523072
:1000E000735044749702000093820201739052305F
:1000F00073500018970200009382420273905230AE
:100100009B021000939252039382F2FF7390023B82
:100110009302F0017390023A73504030970200004E
:1001200093824201739052307350203073503030BC
:100130009301000097020000938202ED7390523009
:10014000130510001315F501635C05000F00F00F97
:10015000930110009308D005130500007300000000
:1001600093020000638A020073905210B7B200003D
:100170009B829210739022307350003097020000DF
:100180009382420173901234732540F17300203042
:1001900093012000930000001301000033B72002F8
:1001A000930300006310774E93013000930010001A
:1001B0001301100033B72002930300006314774C3F
:1001C00093014000930030001301700033B7200208
:1001D000930300006318774A9301500093000000D6
:1001E0003781FFFF33B7200293030000631C774879
:1001F00093016000B70000801301000033B72002B4
:10020000930300006310774893017000B7000080EB
:100210003781FFFF33B72002B703FFFF9B83F3FF54
:100220009393F300631077469301E001B7B0AAFA05
:100230009B80B0AA9390C0009380B0AA9390C00016
:100240009380B0AA9390C0009380B0AA37010300B6
:100250001B01D1E733B72002B70302009B83E3EF12
:10026000631277429301F001B70003009B80D0E74F
:1002700037B1AAFA1B01B1AA1311C1001301B1AA27
:100280001311C1001301B1AA1311C1001301B1AAC6
:1002900033B72002B70302009B83E3EF6314773E7A
:1002A000930180009B00D000939000021B01B000DE
:1002B00013110102B3B020029303F0086394703C61
:1002C000930190009B007000939010021B01B000FE
:1002D0001311010233B120029303A0096314713A90
:1002E0009301A0009B00D00093900002B3B01002D5
:1002F0009303900A639870389301B00013020000D2
:100300009B00D000939000021B01B000131101026A
:1003100033B72002130307001302120093022000D8
:10032000E31052FE9303F008631E73349301C00080
:10033000130200009B007000939010021B01B0009C
:100340001311010233B7200213000000130307004A
:100350001302120093022000E31E52FC9303A00933
:10036000631273329301D000130200009B00F0006F
:10037000939000021B01B0001311010233B7200259
:100380001300000013000000130307001302120003
:1003900093022000E31C52FC9303500A6314732E53
:1003A0009301E000130200009B00D0009390000234
:1003B0001B01B0001311010233B720021302120017
:1003C00093022000E31252FE9303F008631C772A85
:1003D0009301F000130200009B0070009390100244
:1003E0001B01B000131101021300000033B72002FB
:1003F0001302120093022000E31052FE9303A0099F
:100400006312772893010001130200009B00F000A3
:10041000939000021B01B0001311010213000000B1
:100420001300000033B720021302120093022000D1
:10043000E31E52FC9303500A6316772493011001C4
:10044000130200009B00D0009390000213000000F4
:100450001B01B0001311010233B720021302120076
:1004600093022000E31052FE9303F008631C7720F0
:1004700093012001130200009B0070009390100272
:10048000130000001B01B000131101021300000053
:1004900033B720021302120093022000E31E52FC25
:1004A0009303A0096310771E93013001130200002B
:1004B0009B00F00093900002130000001300000066
:1004C0001B01B0001311010233B720021302120006
:1004D00093022000E31E52FC9303500A6314771A20
:1004E00093014001130200001B01B000131101022F
:1004F0009B00D0009390000233B720021302120039
:1005000093022000E31252FE9303F008631C771657
:1005100093015001130200001B01B00013110102EE
:100520009B007000939010021300000033B720026C
:100530001302120093022000E31052FE9303A0095D
:100540006312771493016001130200001B01B000D5
:10055000131101029B00F0009390000213000000B1
:100560001300000033B72002130212009302200090
:10057000E31E52FC9303500A631677109301700137
:10058000130200001B01B000131101021300000050
:100590009B00D0009390000233B720021302120098
:1005A00093022000E31052FE9303F008631C770CC3
:1005B00093018001130200001B01B000131101021E
:1005C000130000009B0070009390100213000000C5
:1005D00033B720021302120093022000E31E52FCE4
:1005E0009303A0096310770A93019001130200009E
:1005F0001B01B000131101021300000013000000E2
:100600009B00F0009390000233B720021302120007
:1006100093022000E31E52FC9303500A63147706F2
:100620009301A0019B00F00193900002333110026E
:1006300093030000631871049301B0019B00100044
:100640009390500233B1000293030000631C7102C7
:100650009301C001B3300002930300006394700261
:100660009301D0019B001002939000021B01100126
:100670001311110233B020029303000063147000C1
:10068000631030020F00F00F63800100939111009E
:1006900093E111009308D005138501007300000059
:1006A0000F00F00F930110009308D0051305000010
:0C06B00073000000731000C00000000088
:1010000000000000000000000000000000000000E0
:1010100000000000000000000000000000000000D0
:1010200000000000000000000000000000000000C0
:1010300000000000000000000000000000000000B0
:081040000000000000000000A8
:040000058000000077
:00000001FF
